:030000000219FDE5
:03000B000200AA46
:03002B0002016C63
:03005B000203029B
:030073000202E89E
:1000800002030406080C10182030406080040608A3
:100090000C10182030406080A0C000070F1F3F0DDB
:1000A0000D0403060D0503030202C2AFC0D0C0E079
:1000B000206217E5256002E473E525F4F58A758B67
:1000C00000D262D0E0D0D0D2AF3285268AC262E5BB
:1000D00026F4603C306803207210758B00D0E0D0AD
:1000E000D0C283C294C295D2AF32C283C294C295A9
:1000F000206E13206610740CD5E0FDE57EB5070474
:10010000429021064280758B00D0E0D0D0D2AF3231
:10011000758A00C28DD262210601B9306805206659
:1001200002D28301B9306805206602D29401B93049
:100130006805206602D29501B9C28030680A20663F
:10014000077408D5E0FDD28301B9C28230680A2065
:1001500066077408D5E0FDD29401B9C29730680AE9
:100160002066077408D5E0FDD29501B9C2AFC2ADD3
:1001700053E6EFC0D0C0E0D2D3D2AFC2CEE52A6002
:1001800007207449152A21CD7800790020742EE5C6
:1001900080307E01F430E50278FF53DACF207E0311
:1001A00043DA20307E0343DA10C2D8C271E58030D2
:1001B0007E01F430E50279FFC3E89970CB3061032A
:1001C000752A40207403752A40885FD27020740D10
:1001D000E52B6004152B21DD43DA01C2D820700223
:1001E00021F0A85F206102C27020740221EE8822F3
:1001F0007882B60403852224C3E52594404002D2C8
:100200006420CF0AD0E0D0D043E610D2AD32C2CFC6
:10021000053A7802E52A6005307402152AC3E55FC5
:1002200094014005756200413A756300756C00E504
:10023000622401F56250037562FF7982B7020D30C6
:100240006D1DC3E52294324016854D227982B70395
:100250000E306D0BC3E52294324004798E8722C3A1
:10026000E5239522600840041523416E0523D8CA72
:10027000056CE56C7002156CD56D63756D017805C4
:10028000C3E56C956E4057C3E56C956F50087801D7
:10029000756D030202A2C3E56C9570500578017577
:1002A0006D01C3E5659524401E7982B7040241D3F0
:1002B000206D14852465E56C046003856E6C756D96
:1002C0000175233C0202DEE5652850057565FF4196
:1002D000D3F565E5650470067563FF756CFFD0E0C6
:1002E000D0D043E610D2AD32C2AFC0D053E67FC209
:1002F00060759100855694855795759104D0D0D23C
:10030000AF32C2AF53E6EFC2ADC0D0C0E0C0F0D252
:10031000D3D2AFA8FBA9FCC2D8307102616953DA0D
:10032000CF207E0343DA10307E0343DA20D271E51A
:1003300080307E01F420E502614088278928A14EA3
:1003400053DACF207E0343DA20307E0343DA10C233
:10035000D8C271307402A13A7800E580307E01F491
:1003600030E502A13A885FA12253DACF207E034311
:10037000DA20307E0343DA10C271206102814253D9
:10038000DACF207E0343DA10307E0343DA20C2D86E
:10039000D271885A895BC3E89558F8E99559F97B79
:1003A000007E087A00C3E8948CE994005005755EDD
:1003B000008134882178A2E6A8216055C3E894C85A
:1003C000E994005008E4D2E4FB7A0A810FC3E89470
:1003D00068E994015008E4D2E3FB7A0F810FC3E887
:1003E00094D0E994025008E4D2E2FB7A1E810FC354
:1003F000E894A0E994055008E4D2E1FB7A3C810F2F
:10040000C3E89498E994085008E4D2E0FB7A787E37
:1004100000C3E8955CFCE9955DFD30E70AECF42447
:1004200001FCEDF43400FD755E00C3EC9AED9E50C6
:1004300003755E01885C895D855A58855B59780231
:10044000A122C3E89527F8E99528F9307C02A10696
:10045000307B02A106307A0281FF2075028165E9B6
:10046000FDE8FC8184E9C313F9E813F830790281CF
:0F047000FFE9C313F9E813F830780281FFE9C3FD
:10047F0013FDE813FC20612CC3EC941CED94024097
:10048F0002819BED701EC3EC94C850180529E52915
:10049F0070021529C3E529940A5002A13A755F002D
:1004AF00D270A13AE529600215297400207F0378E4
:1004BF0096E624FAFEE43400FFC3EC9EFCED9FFDAC
:1004CF00500678007900A106C3EC94FFED9400402C
:1004DF000678FF7900A106EC8575F0A4C5F0A2F7A8
:1004EF0033F87900400302052278FF7900020522D4
:1004FF00E9C313F9E813F8307C0EE9600278FFC303
:10050F00E81338F8E43400F9C3E894FFE9940040A5
:10051F000278FF885FD270206102A13A741FF455F0
:10052F002F4BF52FC274EB7002D274752A403074C2
:10053F0003752A0A306102A14E20740353DAFE209C
:10054F007403752B20D0F0D0E0D0D0D2AD43E6109D
:10055F0032790102057E790302057E790A02057E52
:10056F00791E02057E796402057E79C802057E78C0
:10057F0017E4D5E0FDD8FAD9F6227A147B78020574
:10058F00A57A107B8C0205A57A0D7BB40205A57A9E
:10059F000B7BC80205A57902B27DE4C282D5E0FDCE
:1005AF00D294D5E0FDC294D5E0FDD282D5E0FDD244
:1005BF0083E576D5E0FDC2837496D5E0FDD9D9EAFF
:1005CF00F8D5E0FDD8FBDBCEC28222C37C007D00D4
:1005DF0075F00005F0EA33FAEB33FB50F6EB13FB43
:1005EF00EA13FAC3E9FFE8FEE89AF8E99BF9500429
:1005FF00EFF9EEF8B3EC33FCED33FDD5F0DFEDF9A9
:10060F00ECF822E889F08A20D2D4F8A9F07B0030E8
:10061F00F70B7BFFF42401F8E9F43400F9E88520A7
:10062F00F0A4ADF0F8E98520F0A4AFF0FEED2EF9BF
:10063F0074003FFA7C04C3EA13FAE913F9E813F8DC
:10064F00DCF48BF030F70AE8F42401F8E9F4340015
:10065F00F9E889F0C2D4F8A9F0227882B60403022F
:10066F000708C3E55F9419401EE52D540670182046
:10067F006D3678057994E7146007780A146002786C
:10068F0012C3E54198401F306D09856765756CFF92
:10069F00756D01852224E4F545F546F547F548F5D6
:1006AF0049C26D020708D26D7994E7147013E523E0
:1006BF00F43333F913F8E9540104F9E854FE020650
:1006CF00FCE714147014E523F4333333F913F8E90A
:1006DF00540304F9E854FC020704E523F4333333DD
:1006EF0033F913F8E954070404F9E854F8C39440B4
:1006FF00F8E99400F98845894622C3E54113F9E5E5
:10070F004013F8C3E54598F8E54699F9500CC3E84E
:10071F009480E994FF4016020740C3E8947FE99460
:10072F00005003020740787F7900020740788079F4
:10073F00FF884A894B22E54A2547F8E54B3548F9AA
:10074F00854B20E4300701F43549FA30E709C3EA55
:10075F0094F0401502077EC3EA940F500302077E00
:10076F0078FF79FF7A0F02077E780079007AF0C35D
:10077F00E5249564500AC374019524500B02079C1D
:10078F00E54B20E70E02079CE54B30E706884789CB
:10079F00488A492278A4E6FAC3E54A33F8E54B3391
:1007AF00F9D112E930E70BC3E89480E994FF4013C5
:1007BF00E1D6C3E8947FE994005002E1D6787F79BF
:1007CF0000E1D6788079FFE820E715C3E52398F894
:1007DF004009C3E8940140030207FD78010207FDB9
:1007EF00E8F424012523F840030207FD78FF884C25
:1007FF002278A5E6FAA848A949120612E930E70CB3
:10080F00C3E89401E994FF4016020832C3E894FF4D
:10081F00E99400500302083278FF79000208327819
:10082F000179FFE920E715C3E54C98F84009C3E8C3
:10083F00940140030208597801020859E8F4240191
:10084F00254CF8400302085978FF88242278FFC20C
:10085F006420693D206A12D264C3E541940A4009BD
:0E086F00C3E52594405002C26479A1E76023DE
:10087D00E541601F74FF8541F0848539F0306A03CE
:10088D0075F005A4F8C5F0600278FFC3E8956750D0
:10089D0002A867886622C3E5409440E5419401E5CE
:1008AD006650031401B4046002F566227883E6F500
:1008BD0020120F5375E89012056075E890E5E82059
:1008CD00ECFBA8BDA9BE120FED757155757200C375
:1008DD00740013FD7455606613FC74552CFC740084
:1008ED003DFDECFAEDFBC3E89AE99B4014E571245C
:1008FD0055F571E5723400F572EA2CFAEB3DFB808B
:10090D00E5AE71AF72C3E57213F9E57113F8C3E982
:10091D0013F9E813F87A03C3E913F9E813F8DAF7D2
:10092D00AA201A700975710075720002094B1AEA36
:10093D006008EE28FEEF39FFDAF88E718F7222759E
:10094D00E890227883E6FFE5E820ECF7A8BDA9BE84
:10095D000573C3E57394084052757300E9FA79A0E5
:10096D00E76044EA7007E574601B020986C3E895E9
:10097D00746010E5745006600C140209920460F95D
:10098D00020992E574F574C3946D401B7564C0C380
:10099D0094044013756480C39404400B756440C384
:1009AD009404400375640075BB0922EFC394016084
:1009BD001F7455601BC3E894FFE994035012C3E8FC
:1009CD009571E995725009E564600C15640209E4AE
:1009DD00E564F460020564A864C3E524985002A898
:1009ED0024C3E89565400AA865E565F4600385654F
:1009FD006488258826E573B4070375BB102274320D
:100A0D0079A687F0A4C5F0A2F733F8C3E895644042
:100A1D0002A8648822882488258826886722754044
:100A2D00007541F022C2AF75C820A8CCA9CDAA3A55
:100A3D0030CF010A75C824D2AFAB3BAC3C883B89A3
:100A4D003CC3E89BF8E99C206908F93067026147CF
:100A5D0041A4AD3D8A3DF9EA9DFA600478FF79FF26
:100A6D00AE3EAF3F8B3E8C3FC3EC9FFCC3E99CF584
:100A7D0042A83BA93CC3E89EF8E99FF9C3E54113A1
:100A8D00FBE54013FAE82AF540E93BF541500675C0
:100A9D0040FF7541FF41EEAA40AB41AC40AD417EF8
:100AAD00047F02C3EB940440021E1FC3EB94084065
:100ABD00021E1FC3ED13FDEC13FCDEF7C3EA9CFA17
:100ACD00EB9DFBEF6009C3E913F9E813F8DFF7EAD3
:100ADD0028FAEB39FB8A408B4150067BFF8B408B0C
:100AED0041C3EB94025002D2673069047F03611950
:100AFD007892E6FFC3E537948240110FC3E5379432
:100B0D00A040010FC3EF940640027F057E06E5412C
:100B1D00C4540FF9E541C454F0F8E540C4540F280E
:100B2D00F8C3E89EFAE99400FB4009C3EA9402EB8E
:100B3D00940050047A02E4FB6193AA40AB41EBC4EC
:100B4D00FEEAC4540F4EFCC3EA9CFAEB9400FBC3BF
:100B5D00E813C313F8EA28FAEB3400FB8A408B4103
:100B6D00C3EB94024002C2677806EBC4FE7B00EA39
:100B7D00C4540F4EFAC3EA98FA4005C394025002CA
:100B8D007A027892E6FF3060026193855256855362
:100B9D0057D26043E680C3E49AF8E49BF9306702CC
:100BAD00812DE8FAE9FBD3E913FDE813FC8852899E
:100BBD0053C3EF94036038EF20E00DE82CF8E93DC6
:100BCD00F9ECFAEDFB020BE8E828F8E939F9C3E88E
:100BDD002402F8E93400F97AFE7BFFC3EF94034059
:100BED000E8A548B55884E894F8C508D518161885A
:100BFD005489558A4E8B4F8C508D51306920C3E5E9
:100C0D003394034019E542A2E713F8E555F42401A6
:100C1D0038400B20E7087554FFF42401F555816128
:100C2D00E8FAD3E813FC8852C3EF94036020EF2059
:100C3D00E007E82CF8ECFA814DE8282402F87AFE5A
:100C4D00C3EF940340088A54884E8C5081618854B8
:100C5D008A4E8C50E56BC3335002646BF56B30607C
:0F0C6D0002816B753402D26043E680E52D540698
:100C7C006026A840A941C3E913F9E813F8C2AF53A1
:100C8C00E67F759100C3E498F594E499F595759118
:100C9C0004D26043E680D2AF22D265754400752041
:100CAC0000306B03752040020CC4D265754400758E
:100CBC002040306B03752000D2AF7801206722E50D
:100CCC002D54066002C265C3E541940540137802B9
:100CDC009405400878039405400278063069027840
:100CEC000A206019E544601530690AC3E5339403A2
:100CFC004003D53406D2AFD26CA1969173D2AF001B
:100D0C0000C2AF206726E541C3FB940F40027B0F66
:100D1C00EB240530730123306A027428206201230E
:100D2C00F93069027982E58BC39940B50544E59B9E
:100D3C00F45440B52002A18030690A08C3E8940A33
:100D4C0040010881ED20650281C4C26553E67F75C0
:100D5C0091003067107594007595FE759104D26002
:100D6C0043E68081C4AE40AF41C3E49EF594E49F5A
:100D7C00F595A167C3E5339402500281C430650236
:100D8C0081C4D802A19481EDC26C53E67F759100A9
:100D9C00855494855595759104854E56854F57D23B
:100DAC006043E680D2AFE52D54066008206A020548
:100DBC0033020DD0306C0D206B0A206507158115A0
:100DCC008102162D2278003064053065027801E529
:100DDC003775F007A4F9E5F028F5F0E9A2F013A2B5
:100DEC00F113A2F213F537C394785003753778C317
:100DFC00E53795384008D266C283C294C2953060FC
:100E0C0002C10A855056855157D26043E680222094
:100E1C007D11C2AF754302C282D280D2AF759F439F
:100E2C00020FEAC2AF754302C282D297D2AF759F4E
:100E3C0043020FEA307243207D20C2AF754303900A
:100E4C00014A757E04C295C297306204D294C15E89
:100E5C00D282D2AF759F53020FEAC2AF7543039093
:100E6C00014A757E04C283C280306204D294C17E72
:100E7C00D282D2AF759F33020FEA207D17C2AF75B5
:100E8C004303900125C295306202D294D2AF759F74
:100E9C0053020FEAC2AF754303900125C28330623F
:100EAC0002D294D2AF759F33020FEA207D11C2AFEC
:100EBC00754304C280D297D2AF759F33020FEAC23A
:100ECC00AF754304C297D280D2AF759F53020FEA1D
:100EDC00307243207D20C2AF754305900139757E79
:100EEC0001C294C282306204D283C1FAD280D2AFE2
:100EFC00759F43020FEAC2AF75430590015B757E87
:100F0C0080C294C282306204D295E11AD297D2AFD9
:100F1C00759F43020FEA207D17C2AF754305900100
:100F2C001BC294306202D283D2AF759F43020FEA88
:100F3C00C2AF75430590012FC2943062EBD295D2AB
:100F4C00AF759F43020FEA207D11C2AF754306C2F5
:100F5C0097D282D2AF759F53020FEAC2AF75430688
:100F6C00C280D282D2AF759F33020FEA3072422018
:100F7C007D20C2AF75430190015B757E80C283C238
:100F8C0080306204D295E196D297D2AF759F33022E
:100F9C000FEAC2AF754301900139757E01C295C24B
:100FAC0097306204D283E1B6D280D2AF759F53E101
:100FBC00EA207D16C2AF75430190012FC2833062C7
:100FCC0002D295D2AF759F33E1EAC2AF754301905F
:100FDC00011BC295306202D283D2AF759F53C26699
:100FEC0022900119757E00C283C294C295C280C240
:100FFC0082C297C26222788076070876070876014B
:10100C000876040876FF0876FF0876090876020849
:10101C007601087601788C76010876000876B4089B
:10102C0076FF0876FF0876FF0876030876FF0876C9
:10103C00010876FF0876250876D00876780876C8F9
:10104C000876040876FF08760108760008767A0898
:10105C00760A0876010876010876000876FF227871
:0F106C0087E6FFC272BF0302D2727888C27DE6A8
:10107B0030E102D27DC27E7889E630E102D27EC3B6
:10108B00EF94026008758E01D27302109D758E006D
:10109B00C273227880E6149000809378A4F678814E
:1010AB00E6149000809378A5F67886E61490008D70
:1010BB009378A6F6789FE6F8700108C3E894114080
:1010CB00027811E82828F56E256E256E28F56F2518
:1010DB006E2828F570789CE67538FF75390CB402CC
:1010EB00067538A075390AB403067538827539054B
:1010FB0078A3E61490009A93F569120FED22D28132
:10110B00789DE66002C281227896E6FA7897E6FB34
:10111B007888E6B40305C3EB940EFB307F047A00AA
:10112B007BFFC3EB9AFCC3948250027C82757500E3
:10113B000575EC8575F0A4C3E5F0947D40F222D2E1
:10114B007F311312056F7A007B007C10120565E569
:10115B005F2AFA74003BFBDCF37C04C3EB13FBEA62
:10116B0013FADCF7FEC27F311322E5EF20E603759D
:10117B0020000520903FFFE520146006901DFF1412
:10118B0060009304600375EF1253D9BF7581C043A0
:10119B00FF8012056075EF0243B203E5B324042010
:1011AB00E70DF521E5E320E0068521B343E30112CA
:1011BB000FED7580F075A40F75F13F75D4DF759049
:1011CB004F75A5B075F2F575D50075A60175E241A1
:1011DB00E4F8F6D8FD756B01110212167578988636
:1011EB0076753001C2AF12057912058912056F129F
:1011FB00059012056F12059712056F1217971205BE
:10120B0079120579120574C2AF78FA79FA3085072D
:10121B00D9FBD8F7021C00116B119E3109311378E1
:10122B00988676120FED75885075891275C82475DE
:10123B00910475D84075A82275B80275E690759B18
:10124B0080759D0075D10E75BC5875BB0975BA11AB
:10125B0075E880120560D2AF1208B953DACF207E41
:10126B000343DA20307E0343DA1043DA01C2D8C2DB
:10127B0071120579D2617B037A0CE55E70077A0CEB
:10128B00DB0302121212056F207003021212C270DE
:10129B00E55FC3940240E1E52F541F856160F56162
:1012AB00B560D5DAD5C26153DACF207E0343DA209D
:1012BB00307E0343DA10C2D8C27178A2E67008D22E
:1012CB0074E52F54E0F52FC27575290012057430A3
:1012DB007409C3E529940A4002D275120565780298
:1012EB003074027800C3E55F9840F0C2AF120589F5
:1012FB00120589120589D2AF120579754D001205B9
:10130B0065788CE6C3940150030213DFE530C39478
:10131B000150030213DF207435C3E55F94FF5003C4
:10132B000213DFC2AF12059ED2AF120574C3E55F85
:10133B00940150EFC2AF12058912056A120589D2CA
:10134B00AF120574C3E55F94FF40E902181C7F05DB
:10135B00D27F3113120574C2AFC27F3113AE5FC39C
:10136B00E55F947FD2AF4076120560C2AF12059E47
:10137B00D2AFDFDC314AC3EE94057897F6120579CC
:10138B001216B612179F7F0AD27F3113120574C241
:10139B00AFC27F3113AE5FC3E55F947FD2AF50E630
:1013AB00120560C2AF12058912056A120589D2AF08
:1013BB00DFD6314AEE24057896F61205791216B669
:1013CB001217CE1205743113C3E55F94FF500261FF
:1013DB002102181CC3E55F954D4003855F4D120537
:1013EB007478017988E7B403027805C3E55F984008
:1013FB00026109C2AF12059E12059E12059ED2AF65
:10140B00120579753000E4F531F5320531E531F42B
:10141B0070390532789AE6781914601278321460B4
:10142B000D787D14600878FA146003753200C3E5FB
:10143B003298401715327531B478998676C2AF124F
:10144B00059ED2AF7898867612057412056AE52A46
:10145B007005307402411278012074027806C3E5DE
:0E146B005F9840A7120574E52A700302121262
:10147900C2AF120FEDE4F522F523F524F525F52683
:10148900F56AD2AF7885E6C333F568E4F545F546E4
:10149900F547F548F549F573F52CF52DF5377573CD
:1014A9000875BB1012056012094CE5E820ECFBA891
:1014B900BDA9BEE97001F8887412095075730875E1
:1014C900BB107887E6FE7602116B7887EEF6C2AF1D
:1014D9007564FF120A0B852264852265852266D20E
:1014E900AF75220175240175250175260185636C87
:1014F900756D017888E6B40307C27D307602D27D26
:10150900D268D269753300120F53120F78120A2B61
:10151900120A32120A2B120A32120A2B021534C28B
:10152900AF116BD2AF75730075BB09120CB61206F9
:1015390069120DD1120E1B120A32120CA5306D035D
:1015490012070920670312085C3067031208A31207
:101559000DD1120E40120A32120CB6306D03120769
:1015690045120DD1120EB7120A32120CA5306D03B5
:101579001207A3120DD1120EDC120A32120CB63068
:101589006D03120800120DD1120F53120A321209FB
:101599004C120CA5120DD1120F78120950120A32F1
:1015A90030692F206B2C85676485676585636C7549
:1015B9006D0179187A0CC3E533994009C269D26A79
:1015C9008A350215DBC3E55F940140030215340235
:1015D9001635306A1B206B18E535147004C26AA1F0
:1015E90028F535C3E55F9401400302153402163529
:1015F900753600C3E5629401400985676585636CAA
:10160900756D01C3E56278FA985021307404E52AB2
:10161900601A78F0306B058567647820C3E54198D6
:101629005002A1340536E55F6002C138753600C243
:10163900AF120FED7887E6FE7602116B7887EEF62A
:10164900E4F522F523F524F525F526F568C268D2D7
:10165900AF120560120FED307406E52A70024112CF
:10166900788DE6C39401400241E68111901A0D7804
:10167900201216F8E520B4A50CA31216F8E520B43B
:101689005A0302169611021216B60216B5901A03DB
:1016990078807B0A1216F8A308DBF9901A0F788C68
:1016A9007B181216F8A308DBF9901A2722C2AF1289
:1016B9001737121711901A00740E1216FDA374042D
:1016C9001216FDA374141216FD901A0378807B0A72
:1016D9001216FCA308DBF9901A0F788C7B181216E6
:1016E900FCA308DBF912174A121728901A2722E4DB
:1016F90093F622E6438F01538FFD75EF0275B7A567
:1017090075B7F1F0538FFE22438F02438F0175EFB6
:101719000275B7A575B7F1901A0DF0538FFC229099
:101729001A0D74A5D1FD901A0E745AD1FD227A3082
:1017390079D07820901A40D1F8E520F709A3DAF793
:10174900227A3079D0901A40E7D1FD09A3DAF9223B
:10175900AB77A878BB01027980BB02027981BB0310
:10176900027982BB04027994BB05027983BB060224
:101779007986BB07027992BB08027987BB0902798E
:101789009CBB0A027988BB0B027989E8F7227C05A0
:10179900120579DCFB22C2AF1205891205901205E8
:1017A9009712059E12056A1205891205901205976E
:1017B90012059E12056A12058912059012059712E3
:1017C900059ED2AF22C2AF12059E1205971205904F
:1017D90012058912056A12059E12059712059012C3
:1017E900058912056A12059E1205971205901205C0
:1017F90089D2AF22AE77AF78C2AF120589120589B7
:1018090012058912056ADEF212059E12056ADFF8D1
:10181900D2AF2212179F1217971217977577017572
:1018290078017579001217FD7C05AD5F120579C342
:10183900ED955F70F5C3E55F9401400AC3E55F94D8
:10184900FF40370218601217591216B612179FC2B5
:10185900AF75EF12121797DCD10579C3E5799403B7
:0F186900500280C11217970578E5771490009F01
:1018780093F808C3E57898500280A81217971217B2
:10188800970577C3E577940C5002809412100212E2
:0A18980016B6C2AF75EF12121797D3
:0319FD000211755F
:101A00000E041407070104FFFF09020101A55A0192
:101A100000B4FFFFFF03FF01FF25D078C804FF01DA
:081A200000FF0A010100FFFFB5
:101A400023416C69676E424C33355023202020209F
:101A500023424C48454C4923463333302320202031
:101A60002020202020202020202020202020202076
:101C0000C2AFC2D353D9BF7581C043B20343FF8073
:101C1000752438752503B1C975EF0275E24043F1AB
:101C20002053A4DF75D400D2857DFA780379E67C51
:101C300010752200752300901DD67B0675249875BB
:101C400025013085028142208508D8FBD9F9DCF7CF
:101C500081B4308508D8FBD9F9DCF781B4B189E4C7
:101C600093A3C39A6004DDC381B4DBDBB17B600264
:101C7000812B7B08E493FAA3B15CDBF87A30B15C8A
:101C8000752200752300B17BEAFCEBFDC3ED94FEE9
:101C9000400EB17B8A278B28ED30E0048A828B834B
:101CA000B17B7AC270D8C3ED94FE601350CEBD00F4
:101CB00025EC60097520007521FF0200008100A855
:101CC00027A9280809D804D90281D3B17FEA89AAB3
:101CD000F281C50D81A0C3ED94035049EDA2E092BD
:101CE000007AC5C3E5829400E583941C50902000DF
:101CF00010438F02438F0175B7A575B7F1F030001F
:101D00001FA827A9280809438F01538FFDD804D99C
:101D100002A12089AAE275B7A575B7F1F0A3A10DBC
:101D2000538FFC817C7AC1BD030CE493A3FAB140CC
:101D3000DCF8B138817C817EAA22AB23B15CEBFA5E
:101D4000EA6222752608C3E52313F523E52213F57D
:101D50002250066323A0632201D526EAB1C9B1C986
:101D600075260AEAF4200102D285300102C285B14B
:101D7000C9C3134002C201D526EB22B17FEAFB2082
:101D80008502A17F308502A184752608AE24AF2587
:101D9000C3EF13FFEE13FEB1CDB1C9C3EA13308513
:101DA000024480FA30E703632201C3E52313F523DD
:101DB000E52213F52250066323A0632201D526D91C
:101DC000E52265236523F52222AE24AF250E0FDE22
:101DD000FEDFFCD20122424C48656C693437316326
:041DE000F3300601D5
:00000001FF
